:1000000000308A004D2800003E30840000080319AB
:1000100018280130A100A001A00B0C28A10B0B286F
:100020004A30A000A00B122800000000800B092815
:100030000034BA0803192128831605108312051409
:10004000252883160510831205100130BE000420F8
:1000500083168510831285100130BE00042083169C
:10006000851083128514BB08031D4C283C08BD0075
:1000700083160511831205110130BE00042083167A
:10008000051183120515C830BE0004203D08103C40
:10009000031D4C284A284C28982884011F308305CA
:1000A00007309F000130A8000230A9000430AA00E8
:1000B0000830AB001030AC002030AD004030AE0056
:1000C0008030AF004030B0002030B1001030B200BE
:1000D0000830B3000430B4000230B5000130B6007F
:1000E000B701A70127080F3C031C9C280830A60075
:1000F000260F7B289A282830270784000008B9009B
:10010000A0002608A100031989280310A00CA10B48
:10011000852820188D2838108E283814003038187B
:100120000130B900BA002608BB002708BC00192816
:0A013000A6037828A70A72286300CE
:02400E00793FF8
:00000001FF
